:10000000962AFF3FFF3FFF3FFF00030E8301B8002A
:100010000408B7000A08B9008A0100308B1A0130C1
:10002000F1007108013A031D1F2800300B1901303F
:10003000F1007108013A031D1F2828200B1139080F
:100040008A0037088400380E8300FF0E7F0E0900F7
:1000500003138312A4032408003A031D662A2630E2
:10006000A400A5032508003A031D41282830A50057
:10007000C5227008A600AC227008A700DE22700816
:10008000A8002908003A031DAE280130AA02031C6B
:10009000AB0300302B06031D4F2800302A06031D3A
:1000A000AE280130AA000130AB002C08003A031D35
:1000B0005F282D08013A031D5F280130AE002C088F
:1000C000013A031D69282D08063A031D69280130ED
:1000D000AF002C08013A031D73282D08053A031DB3
:1000E00073280130B0002C08013A031D7D282D082B
:1000F000043A031D7D280130B1002C08013A031D8C
:1001000087282D08033A031D87280130B2002C08E8
:10011000013A031D91282D08023A031D9128013050
:10012000B3002C08013A031D9B282D08013A031D3A
:100130009B280130B4002D08003A031DAD282C087F
:10014000003A031DA9283508033A031DA828B60361
:10015000AC280930AD00AC03AE28AD03FF288617EC
:100160000617861606168615061586102729861385
:10017000061786160612861106118610272986177D
:100180000617861206168615061186142729861765
:100190000617861606168611061186142729861359
:1001A0000617861606128611061586142729861745
:1001B0000613861606168611061586142729861339
:1001C0000613861606168615061586142729861721
:1001D000061786160612861106118610272986171D
:1001E00006178616061686150615861427298617FD
:1001F00006178616061286110615861427292D085D
:10020000003A0319AF282D08013A0319B7282D0821
:10021000023A0319BF282D08033A0319C7282D08ED
:10022000043A0319CF282D08053A0319D7282D08B9
:10023000063A0319DF282D08073A0319E7282D0885
:10024000083A0319EF282D08093A0319F7286029FD
:1002500007148714071587150716871607137C29B7
:1002600007108714071587110712871207137C29B7
:1002700007148714071187150716871207177C299B
:1002800007148714071587150712871207177C298B
:1002900007108714071587110712871607177C297F
:1002A00007148710071587150712871607177C296B
:1002B00007108710071587150716871607177C295B
:1002C0002C08003A031928292C08013A031930296F
:1002D0002C08023A031938292C08033A031940293B
:1002E0002C08043A031948292C08053A0319502907
:1002F0002C08063A031958294A2A85120130A90008
:10030000AF01B101B301B001B201B401AE010130DE
:10031000AA000130AB002630A4000330B600AD01C6
:100320000630AC002808013A031D9929A8010130C4
:10033000B500662A8512A9012F08013A031DA429D8
:10034000AF010430B500662A3108013A031DAC291B
:10035000B1010530B500662A3308013A031DB429FE
:10036000B3010630B500662A2E08013A031DBC29E8
:10037000AE010330B500662A2808013A031DC429DE
:10038000A8010230B500662A2608013A031DCB29D0
:10039000A601B501662A662A85120130A900270840
:1003A000013A031DD729A7010130B500662A2608A6
:1003B000013A031DDE29A601B501662A662A8516C3
:1003C000A901AE013608003A031DE829B501662AE5
:1003D0002608013A031DEF29A601B501662A662AFF
:1003E0008516A901AF013008013A031DFC29B001AF
:1003F0000130B5008512662A2808013A031D052A36
:10040000A8010230B5008512662A2608013A031DAC
:100410000D2AA601B5018512662A662A8516A9014C
:10042000B1013208013A031D1A2AB2010130B500A8
:100430008512662A2808013A031D232AA8010230E2
:10044000B5008512662A2608013A031D2B2AA6014B
:10045000B5018512662A662A8516A901B3013408FA
:10046000013A031D382AB4010130B5008512662A0D
:100470002808013A031D412AA8010230B50085125F
:10048000662A2608013A031D492AA601B5018512EC
:10049000662A662A3508003A03197D293508013A8B
:1004A00003199A293508023A0319CC293508033A69
:1004B0000319DF293508043A0319F0293508053AEC
:1004C00003190E2A3508063A03192C2A08000130B0
:1004D00003138312AA000130AB002630A400283099
:1004E000A5000630AC000030AD000030B500003093
:1004F000A6000030A7000030A8000130A1000130A4
:10050000A2000130A3000030AE000030AF00003088
:10051000B0000030B1000030B2000030B300003055
:10052000B4000130A9000330B6000800672285013D
:100530008601870180308316810006309F00DF30FE
:10054000850001308600803087008312851281018A
:10055000A0308B00AA2AAB2A00300313831285181F
:100560000130F1007108A0007108003A031DC12A92
:100570002208013A031DC12A2008A2000130F00020
:1005800008002008A200F0010800003003138312C5
:1005900005190130F1007108A0007108003A031D2F
:1005A000DA2A2108013A031DDA2A2008A1000130C5
:1005B000F00008002008A100F0010800013003133A
:1005C00083120505F1007108A0007108003A031DAF
:1005D000F22A2308013A031DF22A2008A300013061
:1005E000F00008002008A300F0010800FF3FFF3FD3
:02400E00723FFF
:00000001FF
